:020000040200F8
:10000000B85101229D820002A9FE000289820002ED
:1000100089820002898200028982000289820002AC
:10002000000000000000000000000000F583000256
:1000300089820002000000008983000261AA000298
:10004000C1850002C1850002C1850002C185000290
:10005000C1850002C1850002C1850002C185000280
:10006000C1850002C1850002C1850002C185000270
:10007000C1850002C1850002C1850002C185000260
:10008000C1850002C1850002C1850002C185000250
:10009000C1850002C1850002C1850002C185000240
:1000A000C1850002C1850002C1850002C185000230
:1000B000C1850002C1850002C1850002C185000220
:1000C000C1850002C1850002C1850002C185000210
:1000D000C1850002C1850002C1850002C185000200
:1000E000C1850002C1850002C1850002C1850002F0
:1000F000C1850002C1850002C1850002C1850002E0
:10010000C1850002C1850002C1850002C1850002CF
:10011000C1850002C1850002C1850002C1850002BF
:10012000C1850002C1850002C1850002C1850002AF
:10013000C1850002C1850002C1850002C18500029F
:10014000C1850002C1850002C1850002C18500028F
:10015000C1850002C1850002C1850002C18500027F
:10016000C1850002C1850002C1850002C18500026F
:10017000C1850002C1850002C1850002C18500025F
:10018000C1850002C1850002C1850002C18500024F
:10019000C1850002C1850002C1850002C18500023F
:1001A000C1850002C1850002C185000239740002C8
:1001B00065750002757600021D770002C185000298
:1001C0009FED0B7B41EC160B9FED0B5B26EE077B47
:1001D000BCEEC77BB8EE474B17EE101AA4EE456B8A
:1001E000FCEEC67B17EE900A704700BFAFF30080AD
:1001F000000000000000F03D000000000000F041A1
:10020000002902D0B0FBF1F0704708B14FF0FF3089
:1002100000F01EB80029F8D00246B0FBF1F000FB58
:1002200011217047002902D090FBF1F0704700289F
:10023000C8BF6FF00040B8BF4FF0004000F008B8F2
:100240000029F4D0024690FBF1F000FB1121704729
:10025000704700BF81F0004102E000BF83F000431F
:1002600030B54FEA41044FEA430594EA050F08BF51
:1002700090EA020F1FBF54EA000C55EA020C7FEA15
:10028000645C7FEA655C00F0E2804FEA5454D4EB92
:100290005555B8BF6D420CDD2C4480EA020281EA5C
:1002A000030382EA000083EA010180EA020281EA94
:1002B0000303362D88BF30BD11F0004F4FEA0131E6
:1002C0004FF4801C4CEA113102D0404261EB4101F5
:1002D00013F0004F4FEA03334CEA133302D052427B
:1002E00063EB430394EA050F00F0A780A4F1010437
:1002F000D5F1200E0DDB02FA0EFC22FA05F2801871
:1003000041F1000103FA0EF2801843FA05F3594156
:100310000EE0A5F120050EF1200E012A03FA0EFCD5
:1003200028BF4CF0020C43FA05F3C01851EBE371FF
:1003300001F0004507D54FF0000EDCF1000C7EEB1C
:1003400000006EEB0101B1F5801F1BD3B1F5001F5A
:100350000CD349085FEA30004FEA3C0C04F1010479
:100360004FEA445212F5800F80F09A80BCF1004FA2
:1003700008BF5FEA500C50F1000041EB045141EA24
:10038000050130BD5FEA4C0C404141EB0101013CED
:1003900028BFB1F5801FE9D291F0000F04BF0146DC
:1003A0000020B1FA81F308BF2033A3F10B03B3F1AE
:1003B00020020CDA0C3208DD02F1140CC2F10C023E
:1003C00001FA0CF021FA02F10CE002F11402D8BF9C
:1003D000C2F1200C01FA02F120FA0CFCDCBF41EA68
:1003E0000C019040E41AA2BF01EB0451294330BD37
:1003F0006FEA04041F3C1CDA0C340EDC04F1140414
:10040000C4F1200220FA04F001FA02F340EA0300EA
:1004100021FA04F345EA030130BDC4F10C04C4F130
:10042000200220FA02F001FA04F340EA0300294610
:1004300030BD21FA04F0294630BD94F0000F83F45A
:10044000801306BF81F480110134013D4EE77FEA3D
:10045000645C18BF7FEA655C29D094EA050F08BF89
:1004600090EA020F05D054EA000C04BF194610466A
:1004700030BD91EA030F1EBF0021002030BD5FEAAE
:10048000545C05D14000494128BF41F0004130BDD6
:1004900014F580043CBF01F5801130BD01F000452A
:1004A00045F0FE4141F470014FF0000030BD7FEA9D
:1004B000645C1ABF194610467FEA655C1CBF0B4698
:1004C000024650EA013406BF52EA033591EA030FAF
:1004D00041F4002130BD00BF90F0000F04BF0021A7
:1004E000704730B54FF4806404F132044FF00005DA
:1004F0004FF0000150E700BF90F0000F04BF002153
:10050000704730B54FF4806404F1320410F00045B8
:1005100048BF40424FF000013EE700BF42004FEAB3
:10052000E2014FEA31014FEA02701FBF12F07F4330
:1005300093F07F4F81F06051704732F07F4208BFE7
:10054000704793F07F4F04BF41F40021704730B5EE
:100550004FF4607401F0004521F000411CE700BF3A
:1005600050EA010208BF704730B54FF000050AE0BD
:1005700050EA010208BF704730B511F0004502D5BE
:10058000404261EB41014FF4806404F132045FEAC0
:10059000915C3FF4D8AE4FF003025FEADC0C18BF69
:1005A00003325FEADC0C18BF033202EBDC02C2F15B
:1005B000200300FA03FC20FA02F001FA03FE40EAED
:1005C0000E0021FA02F11444BDE600BF70B54FF0F1
:1005D000FF0C4CF4E06C1CEA11541DBF1CEA1355CF
:1005E00094EA0C0F95EA0C0F00F0DEF82C4481EA37
:1005F000030621EA4C5123EA4C5350EA013518BF57
:1006000052EA033541F4801143F4801338D0A0FB43
:1006100002CE4FF00005E1FB02E506F00042E0FBF0
:1006200003E54FF00006E1FB03569CF0000F18BFF6
:100630004EF0010EA4F1FF04B6F5007F64F540749E
:1006400004D25FEA4E0E6D4146EB060642EAC62131
:1006500041EA55514FEAC52040EA5E504FEACE2E9E
:10066000B4F1FD0C88BFBCF5E06F1ED8BEF1004FA1
:1006700008BF5FEA500E50F1000041EB045170BD1D
:1006800006F0004646EA010140EA020081EA030161
:10069000B4EB5C04C2BFD4EB0C0541EA045170BD5D
:1006A00041F480114FF0000E013C00F3AB8014F1D7
:1006B000360FDEBF002001F0004170BDC4F1000420
:1006C000203C35DA0C341BDC04F11404C4F12005A1
:1006D00000FA05F320FA04F001FA05F240EA0200FC
:1006E00001F0004221F0004110EBD37021FA04F632
:1006F00042EB06015EEA430E08BF20EAD37070BDEC
:10070000C4F10C04C4F1200500FA04F320FA05F04A
:1007100001FA04F240EA020001F0004110EBD3704C
:1007200041F100015EEA430E08BF20EAD37070BDBC
:10073000C4F1200500FA05F24EEA020E20FA04F395
:1007400001FA05F243EA020321FA04F001F0004144
:1007500021FA04F220EA020000EBD3705EEA430EB5
:1007600008BF20EAD37070BD94F0000F0FD101F0E4
:100770000046400041EB010111F4801F08BF013C1D
:10078000F7D041EA060195F0000F18BF704703F05B
:100790000046520043EB030313F4801F08BF013DE2
:1007A000F7D043EA0603704794EA0C0F0CEA13559E
:1007B00018BF95EA0C0F0CD050EA410618BF52EA58
:1007C0004306D1D181EA030101F000414FF000005E
:1007D00070BD50EA410606BF1046194652EA43066C
:1007E00019D094EA0C0F02D150EA013613D195EAE0
:1007F0000C0F05D152EA03361CBF104619460AD128
:1008000081EA030101F0004141F0FE4141F4700131
:100810004FF0000070BD41F0FE4141F4780170BD21
:1008200070B54FF0FF0C4CF4E06C1CEA11541DBF86
:100830001CEA135594EA0C0F95EA0C0F00F0A7F888
:10084000A4EB050481EA030E52EA03354FEA0131B5
:1008500000F088804FEA03334FF0805545EA1313C8
:1008600043EA12634FEA022245EA111545EA106590
:100870004FEA00260EF000419D4208BF964244F127
:10088000FD0404F5407402D25B084FEA3202B61A46
:1008900065EB03055B084FEA32024FF480104FF41A
:1008A000002CB6EB020E75EB030E22BFB61A75468E
:1008B00040EA0C005B084FEA3202B6EB020E75EB21
:1008C000030E22BFB61A754640EA5C005B084FEA89
:1008D0003202B6EB020E75EB030E22BFB61A754656
:1008E00040EA9C005B084FEA3202B6EB020E75EB61
:1008F000030E22BFB61A754640EADC0055EA060E22
:1009000018D04FEA051545EA16754FEA06164FEA64
:10091000C30343EA52734FEAC2025FEA1C1CC0D110
:1009200011F4801F0BD141EA00014FF000004FF09D
:10093000004CB6E711F4801F04BF01430020B4F15E
:10094000FD0C88BFBCF5E06F3FF6AFAEB5EB030C16
:1009500004BFB6EB020C5FEA500C50F1000041EB13
:10096000045170BD0EF0004E4EEA113114EB5C04E0
:10097000C2BFD4EB0C0541EA045170BD41F48011B3
:100980004FF0000E013C90E645EA060E8DE60CEABB
:10099000135594EA0C0F08BF95EA0C0F3FF43BAFD8
:1009A00094EA0C0F0AD150EA01347FF434AF95EA8F
:1009B0000C0F7FF425AF104619462CE795EA0C0F73
:1009C00006D152EA03353FF4FDAE1046194622E740
:1009D00050EA410618BF52EA43067FF4C5AE50EA1A
:1009E00041047FF40DAF52EA43057FF4EBAE12E70A
:1009F0004FF0FF3C06E000BF4FF0010C02E000BFEB
:100A00004FF0010C4DF804CD4FEA410C7FEA6C5CCD
:100A10004FEA430C18BF7FEA6C5C1BD001B050EA70
:100A2000410C0CBF52EA430C91EA030F02BF90EA5B
:100A3000020F0020704710F1000F91EA030F58BF1A
:100A4000994208BF90422CBFD8176FEAE37040F07C
:100A5000010070474FEA410C7FEA6C5C02D150EA1A
:100A6000013C07D14FEA430C7FEA6C5CD6D152EAD5
:100A7000033CD3D05DF8040B704700BF844610469A
:100A800062468C461946634600E000BF01B5FFF799
:100A9000B7FF002848BF10F1000F01BD4DF808ED69
:100AA000FFF7F4FF0CBF012000205DF808FB00BF3A
:100AB0004DF808EDFFF7EAFF34BF012000205DF894
:100AC00008FB00BF4DF808EDFFF7E0FF94BF0120E1
:100AD00000205DF808FB00BF4DF808EDFFF7CEFFE2
:100AE00094BF012000205DF808FB00BF4DF808ED21
:100AF000FFF7C4FF34BF012000205DF808FB00BFF2
:100B00004FEA410C7FEA6C5C02D150EA013C0AD109
:100B10004FEA430C7FEA6C5C02D152EA033C02D1FB
:100B20004FF0000070474FF0010070474FEA41025C
:100B300012F5001215D211D56FF47873B3EB62522F
:100B400012D94FEAC12343F0004343EA505311F056
:100B5000004F23FA02F018BF404270474FF00000E8
:100B6000704750EA013005D111F0004008BF6FF026
:100B7000004070474FF00000704700BF4A0011D29C
:100B800012F5001211D20DD56FF47873B3EB6252E7
:100B90000ED44FEAC12343F0004343EA505323FAF3
:100BA00002F070474FF00000704750EA013002D168
:100BB0004FF0FF3070474FF0000070474FEA41029E
:100BC000B2F1E04324BFB3F5001CDCF1FE5C0DD9AB
:100BD00001F0004C4FEAC0024CEA5070B2F1004FF5
:100BE00040EB830008BF20F00100704711F0804FF8
:100BF00021D113F13872BCBF01F00040704741F4BD
:100C000080114FEA5252C2F11802C2F1200C10FAC0
:100C10000CF320FA02F018BF40F001004FEAC123A4
:100C20004FEAD32303FA0CFC40EA0C0023FA02F348
:100C30004FEA4303CCE77FEA625307D150EA01331E
:100C40001EBF4FF0FE4040F44000704701F00040EE
:100C500040F0FE4040F40000704700BF4FF0FF3C02
:100C600006E000BF4FF0010C02E000BF4FF0010CA6
:100C70004DF804CD4FEA40024FEA41037FEA226C6F
:100C800018BF7FEA236C11D001B052EA530C18BF91
:100C900090EA010F58BFB2EB030088BFC81738BFF6
:100CA0006FEAE17018BF40F0010070477FEA226CE4
:100CB00002D15FEA402C05D17FEA236CE4D15FEAE0
:100CC000412CE1D05DF8040B704700BF8446084614
:100CD0006146FFE70FB5FFF7C9FF002848BF10F1D5
:100CE000000F0FBD4DF808EDFFF7F4FF0CBF01201A
:100CF00000205DF808FB00BF4DF808EDFFF7EAFFA4
:100D000034BF012000205DF808FB00BF4DF808ED5E
:100D1000FFF7E0FF94BF012000205DF808FB00BF53
:100D20004DF808EDFFF7D2FF94BF012000205DF8D9
:100D300008FB00BF4DF808EDFFF7C8FF34BF0120E6
:100D400000205DF808FB00BF4FEA40024FEA410374
:100D50007FEA226C02D15FEA402C08D17FEA236C43
:100D600002D15FEA412C02D14FF0000070474FF0F2
:100D7000010070477BB972B90029BEBF00204FF057
:100D8000004106E008BF00281CBF6FF000414FF093
:100D9000FF30FFF75DBAADF1080C6DE904CE002914
:100DA00009DB002B1ADB00F065F8DDF804E0DDE973
:100DB000022304B07047404261EB4101002B1BDB72
:100DC00000F058F8DDF804E0DDE9022304B0404209
:100DD00061EB4101524263EB43037047524263EBC4
:100DE000430300F047F8DDF804E0DDE9022304B036
:100DF000404261EB41017047524263EB430300F014
:100E000039F8DDF804E0DDE9022304B0524263EB77
:100E10004303704753B94AB9002908BF00281CBFD3
:100E20004FF0FF314FF0FF30FFF712BAADF1080C71
:100E30006DE904CE00F01EF8DDF804E0DDE90223E0
:100E400004B07047024608B50B4643EC172BB5EECD
:100E5000C07BF1EE10FA03D4BDE80840FFF7B0B94B
:100E6000B1EE477B51EC170BFFF7AAF9404261EB5B
:100E7000410108BD2DE9F04786468C460846089E8C
:100E8000154674461946002B40F0C1808542B2FADF
:100E900082F245D94AB1C2F1200300FA02FC954022
:100EA00094402EFA03F343EA0C0C4FEA154EA8B215
:100EB000230CBCFBFEF80EFB18CC08FB00F943EA40
:100EC0000C43994528D9EB1808F1FF3704D299450E
:100ED00002D9A8F102072B44A3EB0903A4B2B3FB88
:100EE000FEFC0EFB1C330CFB00F044EA0344A04262
:100EF00014D92C190CF1FF3304D2A04202D9ACF161
:100F000002032C44241A43EA07401EB1D4400023B4
:100F100034607360BDE8F0874746DDE76346F1E77C
:100F200092BB431B01214FEA154EAFB2200CB3FB1D
:100F3000FEFC0EFB1C330CFB07F840EA034398450C
:100F400061D9EB180CF1FF3004D2984502D9ACF10D
:100F500002002B44A3EB0803A4B2B3FBFEFC0EFB80
:100F60001C330CFB07F744EA0344A7424DD92C1964
:100F70000CF1FF3304D2A74202D9ACF102032C4496
:100F8000E41B43EA0040C0E7C2F1200395409440CF
:100F900020FA03F12EFA03F34FEA154E9040AFB258
:100FA0000343B1FBFEFC0EFB1C10190C0CFB07F8F5
:100FB00041EA0041884522D969180CF1FF3004D27A
:100FC000884502D9ACF102002944A1EB08019BB28B
:100FD000B1FBFEFC0EFB1C110CFB07F743EA0143BF
:100FE0009F420ED9EB180CF1FF3104D29F4202D977
:100FF000ACF102012B44DB1B41EA004193E7604660
:10100000E3E76146F7E76046A4E76346B8E7834253
:1010100006D916B9002108467CE7C6E900E0F9E7E1
:10102000B3FA83F78FB9834201D3724508D8BEEB78
:10103000020460EB030301209C461EB9002169E70E
:101040003846FAE7C6E9004CF8E7C7F1200CBB4088
:101050000EFA07F522FA0CF42EFA0CF1BA401C43F2
:1010600020FA0CF3B8404FEA144901431FFA84FEFA
:10107000B3FBF9F809FB18300B0C08FB0EFA43EA36
:1010800000439A4540D9E31808F1FF3004D29A454D
:1010900002D9A8F102002344A3EB0A0389B2B3FBEF
:1010A000F9F809FB183308FB0EFE41EA03418E45AF
:1010B0002CD9611808F1FF3304D28E4502D9A8F16A
:1010C0000203214443EA0040A1EB0E01A0FB029879
:1010D0004145CE46434602D306D14D4504D20138A0
:1010E000B9EB020E68EB0403002EA7D0B5EB0E029D
:1010F00061EB030101FA0CFC22FA07F3F9404CEA18
:101100000303C6E9003199E74046C5E74346D9E7FE
:1011100010F8012B11F8013B012A28BF9A42F7D0A1
:10112000D01A7047034611F8012B03F8012B002A4F
:10113000F9D17047034613F8012B002AFBD1181A86
:1011400001387047000000002DE9F047044688464A
:1011500017468AB00FF0FAFF0A220023FFF75AFE63
:10116000B8F1010F06460D4608D1CDE900012A4A23
:10117000082120460DF00EFE002012E07F6827486F
:101180003946FFF7C5FF78B139462548FFF7C0FF5C
:1011900050B120463B460121224A0DF0FBFD6FF085
:1011A00004000AB0BDE8F087304619A3D3E9002354
:1011B0002946FFF7DFFD06460D46104619461A4A36
:1011C0000023FFF7D7FD80460F46104619464EF61E
:1011D00060220023FFF7CEFD82468946104619465D
:1011E0004FF47A720023FFF7C5FDCDE904A9CDE9DC
:1011F0000601CDE9082308212046CDE90287CDE983
:1012000000650A4A0DF0C6FDB6E700BFAFF30080E7
:10121000005C260500000000D93D0102EA3D010204
:10122000ED3D0102F63D010280EE36000D3E010269
:10123000A0F101000028FBD1704700BF00000000B2
:101240002DE9F843D0ED037A9846B8EE677B9FED21
:101250002C5B846887EE053B089D1746D0F81490F8
:101260000E46D0ED047A08F051FEE31CB8F1000FF1
:1012700004F1020408BF1C4620FA08F006EB440300
:10128000B8EE677BB3FBF0F387EE056B07EE903AA1
:10129000B8EE675B35EE034BB7EE002B34EE064B32
:1012A0003C4482EE047BB4FBF0F4BCEEC77B07EE5B
:1012B000904A36EE036B85ED007AB8EE677B36EE2A
:1012C000055B37EE037B87EE056B9FED0F7B26EE0C
:1012D000077BFCEEC77B17EE900AA0EB090248459E
:1012E000A9EB000388BF1346B3FBF9F3C5E9010876
:1012F000F61B2F61EE606B61BDE8F883AFF30080F1
:101300000000000065CDCD41000000000000594004
:101310002DE9F04F2DED028B83689DB00C46D0E98E
:101320000375069306469146D0F814A008F0EEFD2A
:101330007B4B09909C4205D07A4B9C4202D07A4B61
:101340009C4256D1069B182203F101084FEA48033C
:1013500007930AAB0021184610F022FB00230090EF
:10136000424630460799FFF76BFF07EE904AB7EE0B
:10137000006BB8EEE77B86EE078B07EE907A9FED69
:10138000665BB8EE676B86EE057B06EE905AB8EEAC
:10139000666B86EE054B37EE047B002738EE478BF5
:1013A000069B03F1030B099BFB4006EE103A4FEA44
:1013B0004B0307EE103AB8EE466BB8EE477B16EEDD
:1013C000087BBAFE477BFCEEC77B17EE904A3E2CAB
:1013D00002D8079BA34228D90137082F1ED10D9BA5
:1013E00089F802300E9B89F801300C9B89F8003097
:1013F0000FE04E490B685B070BD04D4B0122039366
:101400004C4B0494029300231846CDE900330FF0AF
:101410007EF81DB0BDEC028BBDE8F08F069B012F5E
:1014200003F1020308BF9B46BDE7642304FB0AF5F2
:10143000B5FBF3F510AB45454FF018024FF0000136
:10144000184638BF454610F0ABFA3B4600902A4696
:1014500021463046FFF7F4FE119B0893089B9A45FE
:1014600010D3089B9A4531D8DDE9132313431F2B72
:10147000B2D80AAC10AD0FCD0FC495E8030084E8D4
:101480000300ACE7013DA845EBD8631B1F2BE8D850
:101490001822002116A810F083FA16AB2A460093F2
:1014A00021463B463046FFF7CBFE1B9A159B9A42DE
:1014B000D7D20DF1400C0DF1580EBEE80F00ACE88C
:1014C0000F009EE803008CE80300C7E70135AC423B
:1014D000CAD31F2DC8D8631B9845C5D81822002130
:1014E00016A810F05DFA16AB2A46009321463B463B
:1014F0003046FFF7A5FE1B9A159B9A42B4D20DF118
:10150000400C0DF1580EBEE80F00ACE80F009EE84D
:1015100003008CE80300A4E70000000065CDCD4186
:10152000801A060040420F00A0860100D00300226E
:101530000B600102E85D01022DE9F84F8146884603
:1015400000232DED028B19F803605A1C202E00F0A9
:101550006881A6F10901042940F263812B2E15460A
:1015600032D02D2E35D0042446F02003692B4BD0E9
:101570006E2B55D000224FF00A0A944613461046AF
:10158000114614F4006E51D046F02007A7F1610B0C
:10159000BBF1050F4AD8573FFFB2BA454BDC46F0C6
:1015A000200604F08007782E40F0CD80002F00F058
:1015B000CA8050EA010A40F0C68044F4006E4FF041
:1015C000100A1FFA8EFE45E0042419F802609D1CE3
:1015D000CAE74424F9E719F80520681C42F0200204
:1015E0008A4221D0984A934215D000259FED908BD6
:1015F000B8F1000F02D04D44C8F80050B0EE480BCF
:10160000BDEC028BBDE8F88F9FED8B8B8F4B13F8F1
:10161000011B0029DFD16306EAD5B1EE488BE7E76D
:101620009FED878B8A4BF2E70546F0E7A6F130077E
:10163000FFB257452DDA44F0800E14F4807F04F495
:1016400000761FFA8EFE0AD0002F18BF43F0010368
:1016500006B9013219F805607446013591E706B103
:10166000013AAAFB00060AFB0161381841F10001AA
:1016700050EA0106EED0BAF10A0F0CF1010C0CBFD2
:1016800010260F26B445E5DD44F4C07E1FFA8EFE19
:10169000E0E7FE2F83D1A70552D514F08006A4D031
:1016A00050EA010605F1FF3500F0B880260540F14B
:1016B000A2803632B1F5800FC0F08280654FB1F55F
:1016C000000F80F08280BA427FDB0343084603F0BC
:1016D0000306032E03D003F00606062E7ED1043344
:1016E00041F10000B0F5000F78D30132B2F5806F00
:1016F00080F2918000234FF4801102F2FF3221F436
:1017000080111E4641EA025747EC186BB0EE480BB9
:101710000CF056FB0138022804D84F4B222210F05F
:1017200025FA1A50B0EE480B0CF04AFB013802289B
:101730003FF671AF484B222210F018FA1A506AE7B0
:1017400044F4007EA2E71FFA87FA002F6BD0BEF1A7
:10175000000F0CBF65277027BE42A1D119F80560A4
:101760006F1C2B2E04D02D2E24D144F48064A4B2FF
:1017700019F80760A6F13007092F91D8AF1C3D4634
:1017800040F2D34A00274FF00A0B5745DCBF303EEA
:101790000BFB076719F805600135A6F1300EBEF1A5
:1017A000090FF2D9660548BF7F42260548BF92005F
:1017B0003A4475E7A6F1300EBEF1090FDFD96FE7A5
:1017C000001802F1FF32494174E7460800F00100B9
:1017D000013246EAC1764908304370E7B2F5806FBE
:1017E00019DA9B08B0F5800F4FEA900143EA807345
:1017F00083D2002285E70CEB020313F5A27F07DDFD
:10180000B3F59B7F07DA00F02BF8B0EE408B89E749
:101810009FED078B86E79FED088B83E79FED048B99
:10182000F9E613468FE69FED028B5546E0E600BFD2
:101830000000000000000000000000000000F07F39
:10184000000000000000F87F627301025F73010274
:101850005C73010202FCFFFF1400000000000000A6
:101860002DE9FF47804616460F46002900F0A2806A
:10187000B1FA81F4341B002E04F10A04C0F2A280F4
:1018800030460CF081F9044430460CF083F9A4EBA7
:1018900006090546694630460CF0A4F9A9EB050394
:1018A0006A4640467D3339460FF02CFFA6428246F9
:1018B0000D4600F38380B9F13F0F00F381804FF0B4
:1018C000FF33A9F12000C9F1200103FA00F003FA67
:1018D00009F223FA01F103FA09F3024328EA0303A8
:1018E0000A4327EA020213430CBF01200020002D07
:1018F00000F08A80B5FA85F3E31A40F2FE7203F233
:101900003E43934200F38980002B23EAE376D4BF61
:1019100001223246121BA2F23341A2F23447A2F254
:101920005344C1F1200C2AFA01F325FA04F4C7F15B
:10193000200E05FA0CFC25FA01F105FA0EFE43EA29
:101940000C03A2F2544CA2F2544223432AFA07F4A5
:1019500025FA0CFC44EA0E0444EA0C04C7F1200CFE
:1019600014F0010F54D0A8B14FF0FF3000FA02F28A
:1019700000FA07F4144320FA0CF2B840144303F0C1
:1019800001022AEA000A25EA04054AEA020A5AEA9A
:10199000050A3DD0013341F10002C2F3130253EABC
:1019A000020138D0184642EA065141EC100B04B04F
:1019B000BDE8F087B0FA80F420345BE7012096E7B9
:1019C000002094E7C6F1000948460CF0E3F8241A19
:1019D00048460CF0DFF8A61B0546694648462E44EB
:1019E0000CF072F96A46404606F17C0339460FF066
:1019F00089FE82460D46404639460CF0DBF88145AB
:101A00008CBF0020012072E7BAFA8AF3203373E713
:101A1000C1F31302C6E70136C4E79FED010BC6E729
:101A2000000000000000F07F10EE902A764922F0BE
:101A300000438B4217D975498B4203D805D110EE6C
:101A4000103A13B130EE000B7047002A9FED500B97
:101A500004DD9FED517B37EE000B70479FED507B0F
:101A600037EE400B70476A498B4212D8A1F1DE7104
:101A70008B420BD8B7EE006B9FED4B7B30EE077BB4
:101A8000B4EEC67BF1EE10FA00F381804FF0FF3325
:101A900015E06049B0EEC07B8B424FD8A1F55021D4
:101AA000B7EE006B8B4241D837EE075B002335EE73
:101AB000465BB0EE006B37EE067B85EE070B591CDC
:101AC00020EE005B9FED3A7B9FED3B4B25EE056BD7
:101AD0009FED3B3B06EE074B9FED3B7B04EE067B09
:101AE0009FED3B4B07EE064B9FED3B7B04EE067BE9
:101AF0009FED3B4B07EE064B9FED3B7B16EE073B06
:101B00009FED3B7B13EE067B9FED3B3B17EE063BC9
:101B10009FED3B7B13EE067B27EE067B04EE057BF9
:101B200027EE007B1FD130EE470B704737EE465B48
:101B3000012337EE066B85EE060BC0E736498B4274
:101B40000BD2B7EE085B0223B7EE006B37EE454BC6
:101B500007EE056B84EE060BB1E7BFEE006B0323C7
:101B600086EE070BABE72D49002A2D4801EBC30198
:101B700000EBC30393ED006B37EE467B37EE407B03
:101B800091ED000B30EE470BB8BFB1EE400B704744
:101B9000075C143326A6913C182D4454FB21F93FD1
:101BA000182D4454FB21F9BF9C7500883CE4377E16
:101BB00011DA22E33AAD903FEB0D76244B7BA93F3F
:101BC0009AFDDE522DDEAD3F513DD0A0660DB13FF6
:101BD0006E204CC5CD45B73FFF8300922449C23FDC
:101BE0000D5555555555D53F2F6C6A2C44B4A2BFA1
:101BF0006D9A74AFF2B0B33F711623FEC671BC3F4D
:101C0000C4EB98999999C93FFFFF0F440000F07FFA
:101C1000FFFFDB3FFFFFF23F00800340782D010212
:101C2000582D0102000000007FB58DED000B019BD7
:101C3000214A23F00043934206D89FED1D1B07B0B5
:101C40005DF804EB00F014BA1C4A934204D907B0C3
:101C50005DF804EB00F0F4B902A800F031F800F0F0
:101C6000030001280BD0022812D0C0B99DED041B3F
:101C70009DED020B00F0FCF907B05DF804FB9DED53
:101C8000041B9DED020B00F0DFFCB1EE400BF3E70F
:101C90009DED041B9DED020B00F0EAF9F5E79DEDCB
:101CA000041B9DED020B012000F0CEFCE4E700BF19
:101CB0000000000000000000FB21E93FFFFFEF7F74
:101CC000F0B510EE907A964B89B0064627F00041A9
:101CD000994207D80022002380ED000BC0E90223BF
:101CE00000201BE08F4B99423BD8A3F51B23002F0C
:101CF0009FED7B7BA3F5F06319DD994230EE470B36
:101D00000ED09FED796B30EE467B012030EE470B15
:101D100086ED007B30EE460B86ED020B09B0F0BD80
:101D20009FED737B9FED746B30EE470BEBE79942B1
:101D300030EE070B0ED09FED6C6B30EE067B4FF054
:101D4000FF3030EE470B86ED007B30EE060B86ED64
:101D5000020BE3E79FED667B9FED676B30EE070BB1
:101D6000EBE7714B99426BD8B6EE007BB0EEC00B3F
:101D70009FED636B00EE067BFDEEC77BB8EEE75B85
:101D800017EE900A9FED567B1F2805EE470B9FED3F
:101D9000567B25EE077B30EE476B05DC421E634B1E
:101DA00053F822308B4208D116EE903A0A15C3F34D
:101DB0000A53C3EB1153102B02DC86ED006B1AE0C3
:101DC0009FED4B4B25EE044B30EE446B30EE467BE3
:101DD00037EE447B9FED484B15EE047B36EE474BC8
:101DE00014EE903AC3F30A53D31A312B17DCB0EE3A
:101DF000460B86ED004B96ED006B002F30EE460B48
:101E000030EE470B86ED020B88DAB1EE466BB1EE91
:101E1000400B86ED006B86ED020B40427EE79FEDA6
:101E20003A7B25EE077B36EE470B36EE406B36EEFF
:101E3000477B9FED376B15EE067B30EE476BBCE7BB
:101E40003B4B994206D930EE400B80ED020B80ED02
:101E5000000B45E70A1510EE103A08A8A2F2164248
:101E60001C46A1EB0255032145EC174BBDEEC76B99
:101E70009FED295BB8EEC66B37EE467B8DED026BAE
:101E800027EE057BBDEEC76BB8EEC66B37EE467B23
:101E90008DED046B27EE057B8DED067B30ED027B2F
:101EA0000B460139B5EE407BF1EE10FAF6D0214930
:101EB00002A8019102210091314600F041F9002F62
:101EC000BFF62CAF96ED007BB1EE477B86ED007B35
:101ED00096ED027BB1EE477B86ED027B9DE700BF6E
:101EE00000004054FB21F93F3163621A61B4D03DD8
:101EF0000000601A61B4D03D7370032E8A19A33BB1
:101F000083C8C96D305FE43F0000002E8A19A33BEF
:101F1000C14920259A837B390000000000007041F0
:101F2000FB21E93F7BD90240FB213941AC3601025C
:101F3000FFFFEF7F2C3701027FB58DED000B019B7A
:101F4000234A23F00043934207D800209FED1E1B35
:101F500007B05DF804EB00F077BB1E4A934204D94A
:101F600007B05DF804EB00F06BB802A8FFF7A8FE1D
:101F700000F0030001280CD0022811D0D0B90120B4
:101F80009DED041B9DED020B00F05EFB07B05DF8BC
:101F900004FB9DED041B9DED020B00F069F8F5E7D5
:101FA0009DED041B9DED020B012000F04DFBB1EEF9
:101FB000400BEBE79DED041B9DED020B00F058F884
:101FC000F5E700BFAFF30080000000000000000054
:101FD000FB21E93FFFFFEF7F7FB58DED000B019BFC
:101FE000154A23F00043934207D801209FED101BB0
:101FF00007B05DF804EB00F07FBB104A934204D9B0
:1020000007B05DF804EB00F01BB802A8FFF758FE1C
:10201000400000F002009DED041BC0F101009DEDA9
:10202000020B00F069FB07B05DF804FBAFF3008022
:102030000000000000000000FB21E93FFFFFEF7FF0
:1020400008B52DED028BB0EE408B0BF0B9FE20B938
:1020500038EE080BBDEC028B08BD9FED037B87EECD
:10206000070BF7E7AFF3008000000000000000005E
:10207000B0EE407BB7EE000B17EE901A21F0004156
:10208000B1F1795F39D327EE075B2B4B994227EEED
:10209000017BB6EE006B9FED1C3B9FED1D4B25EECB
:1020A000066B05EE034B9FED1C3B14EE053B9FEDCD
:1020B0001C4B03EE054B9FED1C3B14EE053B9FEDC7
:1020C0001C4B03EE054B24EE054B14EE057B04D8A8
:1020D00036EE477B30EE470B7047184B99420DD8D0
:1020E0000022A1F5001343EC152B36EE456B30EEC4
:1020F000450B36EE476B30EE460B7047B5EE025B94
:10210000F3E700BFAFF30080D43888BEE9FAA8BD7A
:10211000C4B1B4BD9EEE213EAD529C804F7E923E36
:102120009015CB19A001FA3E7751C1166CC1563FEC
:102130004C5555555555A53F3233D33F0000E93F27
:102140002DE9F04F2DED068BADF5137D12F1140F37
:102150009A460F46BE4B6FF01705A2990AF1FF3B56
:10216000A39E0DF1680E53F82190A6BFD31E18212F
:102170000023019009EB0B04A8BF93FBF1F303FBD1
:102180000555A3EB0B009FEDAC6B154406EB800CE3
:102190000022A2420EDD1AAA0DF5D47E002402EB25
:1021A000CA024C4525DCDDF804C0104600219FED35
:1021B000A27B15E0D04209D45CF8221007EE901AF9
:1021C000B8EEE77B0132AEEC027BE2E7B0EE467B95
:1021D000F8E7BCEC025B90ED006B013105EE067B8D
:1021E0005945A0F10800F4DD01340832AEEC027B61
:1021F000D7E706AA06EB83034C4602EB890202935B
:102200009FED8F9B9FED90AB0392E3006AAA21465E
:10221000049392AB02EBC40203EBC40313ED280B4F
:1022200006AB18460029A2F1080249DC28460593AE
:1022300000F07AFBB4EE007BB0EE408B20EE077B23
:10224000BBFE477B002D059BB2EE006B07EE468B75
:10225000FDEEC87B17EE908AB8EEE77B38EE478B31
:1022600040DD611E06AAC5F1180052F8216046FA49
:1022700000F290448240B61A06AA42F82160C5F1E5
:1022800017021641002E3CDD002108F101086FF015
:102290007F4E08468C4267DC002D04DD012D7ED088
:1022A000022D00F08680022E2BD1B7EE000B30EE0F
:1022B000488B30B3284600F037FB38EE408B20E0E7
:1022C00020EE097B0139BDEEC77BB8EEC77B07EE78
:1022D0004A0BBDEEC00BA0EC010A92ED000B37EEED
:1022E000000B9FE705D1621E06A951F82260F61582
:1022F000C8E7B6EE007BB4EEC78BF1EE10FA31DA28
:102300000026B5EE408BF1EE10FA40F0A580621E7B
:1023100000214A4554DA00296DD0013C06AB183D36
:1023200053F82430002BF8D0B7EE000B284600F00D
:10233000FBFA621C6AA9D30001EBC20122469FEDA1
:10234000406B002A80F2B2802246002AC0F2D08080
:102350006AA9DFF800C1002001EBC205A11A9FEDB8
:10236000367BBAE002268FE79C465CF8042B58B90E
:102370007AB10131C2F180728C424CF8042C0CDD30
:10238000DCF8002003F1080CAEEB02024CF8042C40
:1023900001220131634610467CE701207CE7621E82
:1023A00006AB53F82230C3F3160306A941F82230D6
:1023B00079E7621E06AB53F82230C3F31503F4E746
:1023C00006AB53F82230013A1943A2E7013352F821
:1023D000041D0029FAD0049A04EB0A011AAE601C0D
:1023E00002F51272234406EBC1016A44983A834213
:1023F00004DA1C4609E7039A0123E8E7029C019EE0
:1024000054F8204007EE904A04940024B8EEE77B8D
:10241000A1EC027B9FED087B8C465C4503DD01301F
:10242000A2EC027BE3E7B6EC025B3CED026B01340D
:1024300005EE067BF1E700BF000000000000000091
:10244000000000000000703E00000000000070412D
:1024500034380102982D0102B0EE480B684200F0BA
:1024600063FA9FED736BB4EEC60BF1EE10FA17DB57
:1024700006AA18359FED707B20EE077BBDEEC77B6B
:10248000B8EEC75B05EE460BBDEEC00B10EE103A82
:1024900042F82430013417EE103A42F8243043E772
:1024A000BDEEC00B06AA10EE103AF6E706A850F8EB
:1024B0002200013A07EE900A0190B8EEE77B27EE82
:1024C000007B20EE060B21ED027B3AE7BCEC025BC1
:1024D000B5EC026B013005EE067B484501DC81421C
:1024E000F4DA42A8013A00EBC10181ED007B2CE750
:1024F000A29A022A0ADC002A2DDC46D008F0070046
:102500000DF5137DBDEC068BBDE8F08FA29A032A72
:10251000F4D142A9A3F1080220460A44114600283A
:10252000A1F1080152DC21460129A2F108025DDC7B
:1025300042AA9FED437B1344012C67DC9DED425B77
:102540009DED446B002E67D187ED005B87ED026B3C
:1025500087ED047BD2E742AA9FED396B13442246F4
:10256000002A24DA4EB3B1EE467B44AA012387ED5C
:10257000007B9DED427B37EE467B9C4220DA0EB11C
:10258000B1EE477B87ED027BB8E742AA9FED2C7B3B
:102590001344002C05DA0EB1B1EE477B87ED007BCA
:1025A000ACE733ED026B013C37EE067BF1E733ED30
:1025B000027B013A36EE076BD2E7B0EE467BD4E7FA
:1025C000B2EC026B013337EE067BD6E791ED007B70
:1025D00091ED025B013837EE056B37EE467B81EDFE
:1025E000006B37EE057B81ED027B98E792ED007B77
:1025F00092ED025B013937EE056B37EE467B82EDDB
:10260000006B37EE057B82ED027B8DE733ED026BCD
:10261000013C37EE067B8FE7B1EE455BB1EE466BD2
:10262000B1EE477B87ED005B87ED026B90E700BF63
:102630000000000000007041000000000000703E3B
:102640000000000000000000B0EE407B17EE903A62
:1026500023F00043B3F1795F01D200F0F5B920EE29
:10266000005B9FED176B9FED183B20EE054B15EEC1
:10267000063B9FED176B03EE056B9FED173B16EEC8
:10268000053B9FED176B03EE056B40B99FED163BC5
:1026900015EE063B03EE047BB0EE470B704724EECD
:1026A000066BB6EE003B11EE036B16EE051B9FEDBD
:1026B000106B04EE461B30EE410B7047AFF3008009
:1026C0007CD5CF5A3AD9E53DEB9C2B8AE6E55A3EBC
:1026D0007DFEB157E31DC73ED561C119A0012A3F58
:1026E000A6F810111111813F495555555555C53F53
:1026F000495555555555C5BF10EE903A884923F0B8
:1027000000428A4210B533D8FDEEC07B17EE901A16
:10271000002942D1431C10EE104A2343134306D133
:10272000B7EE006BB0EEC07B86EE070B10BD012844
:10273000FCD030EE017BBFEE006B53EC172B86EE26
:10274000074B0A46B7EE006B43EC152B35EE400BFA
:1027500031EE400B53EC142B0A4643EC172B05EEDD
:10276000076B00EE076B06EE047BB0EE470BDDE770
:102770006C498A4211D9002B9FED497BBCBFB1EE59
:10278000400BB1EE411B37EE407B9FED470B30EE27
:10279000410B9FED471B30EE070B20EE006B6149AC
:1027A0008A429FED455B9FED464B26EE067B20EE71
:1027B000063B07EE054B9FED445B9FED452B04EE7A
:1027C000075B9FED454B05EE074B9FED455B04EE28
:1027D000075B9FED454B05EE074B9FED455B07EE15
:1027E000025B9FED452B05EE072B9FED455B02EE4F
:1027F000075B9FED452B05EE072B9FED455B02EE3A
:10280000075BB0EE457BB0EE415B04EE067B07EE66
:10281000035B9FED417B05EE061B03EE071B30EECD
:10282000016B1DD907EE900A26EE064B9B17B8EEFA
:10283000E77B03F00203C3F1010336EE076B84EE7E
:10284000065B35EE416B30EE466B36EE066B37EECF
:10285000466B07EE903AB8EEE70B26EE000B65E705
:1028600001281AD0BFEE007B51EC160B87EE065BF9
:102870000020B7EE006B41EC140B34EE400B31EE50
:10288000401B53EC152B024643EC172B04EE076B51
:1028900001EE076B06EE057B67E7B0EE460B45E7FA
:1028A000182D4454FB21E93F075C143326A6813CD4
:1028B0000000000000000000D47ABF74702AFB3EC4
:1028C000E9A7F0320FB8123F68108D1AF726303F93
:1028D000735360DBCB75F3BE1583E0FEC8DB573F57
:1028E00093846EE9E326823FFE41B31BBAA1AB3F5E
:1028F000A69237A0887E143F0165F2F2D844433F88
:10290000280356C9226D6D3F37D60684F464963F7E
:102910007AFE10111111C13F635555555555D53FDC
:10292000FFFF2F3E2794E53F10EE902AC2F30A5393
:10293000114610B4C3B922F0004210EE103A1A4307
:1029400018D02B4C9FED267BA04220EE070B10EEFB
:10295000902AC2F30A531146A3F136030DDAD00FC1
:102960005DF8044B00F048B840F2FF72934204D186
:1029700030EE000B5DF8044B70474CF25032904241
:1029800004DDC80F5DF8044B00F04AB8184440F26B
:10299000FE739842F5DC00280ADD21F0FF4121F4A6
:1029A000E00153EC102B41EA005343EC102BE1E71C
:1029B00010F1350F01DAC80FD2E721F0FF413630B0
:1029C00021F4E00153EC102B9FED077B41EA00530B
:1029D00043EC102B20EE070BCCE700BFAFF30080D9
:1029E0000000000000005043000000000000903C88
:1029F000B03CFFFF000000009FED050B9FED067B44
:102A0000002800FE077B27EE000B7047AFF3008025
:102A10000000000000001000000000000000108016
:102A20009FED050B9FED067B002800FE077B27EE40
:102A3000000B7047AFF30080FFFFFFFFFFFFEF7F4A
:102A4000FFFFFFFFFFFFEFFF9FED076BB7EE007B80
:102A500082B037EE067B8DED007BDDE9002302B00E
:102A6000704700BFAFF300800000000000001000BE
:102A700070B5ADF50E7D012002A901F0DDF8044628
:102A800020B1014636480BF078FD24E005AE014642
:102A90001023324602980CF016F8044610B1014695
:102AA0003048F0E73378013BDBB2FD2B05D92E48E7
:102AB0000BF063FD6FF001040DE00A22304603A91C
:102AC0000AF000F8039B0546B34208D127480BF0F3
:102AD00054FD6FF0150420460DF50E7D70BD0146C6
:102AE0004FF4805009F09CFE064618B9294620484C
:102AF0000BF043FD2B463246102102980BF0E3FF0A
:102B0000044610B101461B48BDE701464FF405726B
:102B100009A80EF045FF184B18490993184B04AA51
:102B20000A93184B09A80B930123ADF8043001ABAD
:102B3000CDE98B6505F0D8FF044610B10146124877
:102B4000A1E704981149843005F0A0FF014608B9B7
:102B50000F48ADE72246049806F076F8BBE700BFC1
:102B6000F23A0102143B0102323B0102433B0102F3
:102B7000603B01027D3B010271020102E53B010263
:102B80009B020102AF020102A03B0102BE3B010217
:102B9000C33B01027FB50BAB05930393054B0222A8
:102BA000029300231846CDE9003300F0C7FD07B0BB
:102BB0005DF804FBF03B01022DE9F04F91B000936A
:102BC00002F004030293C2F3C2030E4601338107ED
:102BD0000546DDF868900392059340F0BC81041D22
:102BE00030B1072E09D86FF01B0011B0BDE8F08F8F
:102BF00006F00706341DC6F10806009B4FF00008DA
:102C00004FF0040A591E4FF0FF3347460193C34665
:102C10005346CDF810800DB100982060059800282B
:102C200000F3EB809948009A824203D3984882428D
:102C3000C0F0E380039AA4EB050E92074FEA9E00D2
:102C400000F106810F2F00F2B480002D00F0088102
:102C500007F140020DEB020C019A0CF8200C0CF865
:102C6000102C049801300490EAE07A2860D84B28B0
:102C700010D847285CD829282FD8252855D057D8D0
:102C8000A0F12302D2F1000C4CEB020C202818BF5B
:102C9000E34675E04C382E284AD8DFE800F0714949
:102CA000494949494949494949494C494949494991
:102CB0004949495A494C4C5A5A5A714C6E497149C2
:102CC000184C18494983804C49494C4980000020E0
:102CD0004FF0000B4FF0040A39E00122A0F12A0C5A
:102CE0005FFA8CFC02FA0CFC1CEA0E0F48D11CF0B7
:102CF00062502ED11CEA020B42D0013C5444B4FB7A
:102D0000FAF40AFB04F4002D61D0A3EB050CA444F3
:102D1000B4453FF668AF002868D1042B47D159F875
:102D2000043B2360042304342AE0019A013A01920F
:102D30004FF0000B24E011F8010C6C2834D1002076
:102D400011F8023C83466C2BC4D14FF0080A53465D
:102D5000D3E709F1070929F00709073424F007042C
:102D6000F9E802AB35B106982044B0423FF63BAFDC
:102D7000C4E900AB4FF0000B08344FF0080A53468B
:102D800011F8010F002878D0BBF1000F7FF46DAF70
:102D90002528F5D14FF0010B019B013301934FF032
:102DA000040AECE7584693E700208346A5E7082B82
:102DB00002D06FF0150018E709F1070929F007099B
:102DC000B9EC027B84ED007B08230834D8E768B9AE
:102DD000042B02D109F10409A4E7082BE9D109F178
:102DE000070929F0070909F10809EDE705980138F5
:102DF000059059F8040B00900DE7039A900720D531
:102E00004FF0010CA4EB050E4FEA9E00BEF5007FCB
:102E1000CFD20F2FCDD8F5B107F140020DEB020E46
:102E2000019AC0B20EF8200C0EF8102CBCF1000F65
:102E30003FF417AF60F07F000EF8200C08F1010896
:102E40000137C5F108024FF6DA7E0434069297E79F
:102E50004FF0000CDAE7BCF1000F01D00136EFE7CC
:102E6000029A0236002AEBD10098CDE90631FEF72E
:102E700061F9DDE906310644E2E7631BB3F5806FD3
:102E800097D23DB9A6F10804E018AEE6B01B0102E6
:102E900074730102029A9B0828602B709DF8103011
:102EA000C2B1EB7085F80280B8F1000F05D008A818
:102EB000C5F1010C7A1C013A0ED14FF0000AC5F1A0
:102EC00001030DF1200901930DF1300B574511D18C
:102ED000601B8AE66B70E5E710F8013B1906EAD53E
:102EE00004EB0C0EB64503F07F033FF67CAE04F80E
:102EF000013BE0E7B8F1000F03D099F90020002A68
:102F000017DB029BD3B11AF80B2004F8012B002227
:102F1000019B98182044B0423FF665AE99F8000036
:102F2000009904F8010B204603920EF012FD039A5B
:102F300014440AF1010A09F10109C7E799F80020D0
:102F400055F822300093029B009845F82230FEF796
:102F5000F1F8421CDCE76FF00D0046E62DE9F04F7A
:102F60009BB0DDF890B00993CBF3C003044616463E
:102F7000884690F802A00B9341B9457800780AEB97
:102F800080002044454516D8A0EB0408E3780A9356
:102F9000BAF1000F02D01BF0010F15D10A9B002BD4
:102FA00039D11EB141462046099AB04745462846C8
:102FB0001BB0BDE8F08F471C3846FEF7BBF8013068
:102FC000384408F10108DDE7227863680692089327
:102FD000069B92000C9204EB8301002E40F0E680E9
:102FE0000F460026454601EB0A08474522D017F850
:102FF000013B069154F82300FEF79CF8259B0699A7
:10300000013033B1269B9E423EBF259B23F816001C
:1030100001360544E9E71BF0020FC2D023781F46B2
:1030200006939B000C93636804EB87010893002EC2
:1030300056D145461BF0050F01EB0A070CBF4FF0B8
:10304000020A4FF0010A0A9B07EB43090BF0020347
:1030500006934F45ABD017F8021B17F8013C54F804
:1030600023808E4B984502D38D4B984519D30B9BEB
:1030700023B308980BF056FA00B38A48036813F09C
:10308000060F0CD0089B04910393874B01460293D3
:10309000002302221846CDE90033FFF77BFD023DF5
:1030A000D7E70B9B23B108980BF03CFA0028E4D13A
:1030B0001BF0010F05D1A5EB0A05CAE7069B002B03
:1030C000C7D04046FEF736F8259B3BB1269B9E4273
:1030D0003FBF259A431C22F8163001360544B8E755
:1030E000BAF1000F66D01BF0040766D057464FF0C8
:1030F000000916A8524607910EF02BFC079901EB28
:103100000A0307930A9B0A9A5B000E93079B03EB43
:1031100042030D930BF002030F930D9B079A93420A
:103120004DD1002163781BF0020F03EB09004FEA39
:10313000570218BF0A461BF0010FC0B203D11BF0A3
:10314000040F18BF39466070A170E2702046099ADA
:103150000C990893B047051EFFF629AF069B394628
:103160002370089B099A63700A9B84F802A0E3709D
:1031700016A8B047071EC0F28C800C9BA8EB0A0172
:10318000C91A0E9B099A0798C91AB0470028C0F2BD
:1031900082804FF000082F443D180DF1480BC145C7
:1031A00055D80021099A0846B04700E7D1460027C4
:1031B00012A89FE75746D146A1E7B9469FE7079B6C
:1031C00013F8021B13F8015C079354F82520334BC6
:1031D0009A4202D3324B9A4217D30B9B23B10898E1
:1031E0000BF0A0F9002898D10F9BC3B907F1680331
:1031F0007A1C0DEB03001AAB023753FA82F200F887
:10320000101CFFB202F8105C87E70B9B23B10898F3
:103210000BF088F9002880D11BF0010F0AD009F1CA
:10322000680309F101020DEB030909F8205C5FFA5C
:1032300082F972E71BF0040F3FF46FAF07F16803E8
:103240007A1C0DEB030707F8105CD7B265E718F896
:103250000B30259F54F823A08DF847300FB137F875
:1032600018700121099A0DF14700B047002812DBC0
:10327000054427B95046FDF75DFF471CBFB23946EC
:103280005046099AB047002805DB054408F10108BB
:1032900085E73D468BE6054689E600BFB01B010287
:1032A000747301029C030022F03B0102014B186081
:1032B000704700BF0000002270B50446044E451858
:1032C000AC4200D170BD336814F8010B9847F7E7A2
:1032D0000000002280B505460E461746984608F0C5
:1032E000D1FE03460EF042FC0446DFF81890424639
:1032F00049F8003039463046A84754F8090004F030
:10330000E9FF00BF100000000020074B074A1A60C9
:10331000074B084A1860536943F460235361BFF3B5
:103320004F8FBFF36F8F7047240C002200127A007A
:10333000200C002200ED00E02DE9F84F81462E48D8
:103340000F460BF080FA064670B92C4C0546A04695
:103350004FF0010BDFF8A8A0544507D3B9F1000FD7
:1033600002D04FF0010AE5B9BDE8F88F237B6BB1BD
:103370002368DB680BB12046984723681B6943B973
:10338000636804222046196800F096F9013610346B
:10339000E2E7204698470028F2D00BFA06F31D43D7
:1033A000F4E7A94695FAA5F4B4FA84F40AFA04F30A
:1033B000260108EB04146FEA030B25EA0305237BBF
:1033C00063B158F806301B698BB946447368042210
:1033D0002046196809EA0B0900F06EF9002DE1D1C9
:1033E0001FB16420002108F003FE4D46BBE72046D4
:1033F00098470028F2D1E8E7300C0022882101022A
:103400009821010208B5034608462BB1044A13600F
:1034100000F0FAFB002008BD6FF01500FBE700BFCD
:103420000400002208B50023074A4FF47A71137094
:10343000064A07481360074A1360FFF7E3FFBDE839
:10344000084000F085B800BF1C200022280C002294
:1034500037E800022C0C002270B50B4D297841B9D9
:103460000120FFF769FF094C094EB44202D3012342
:103470002B7070BD63685B791BB1236820469B6825
:1034800098471034F1E700BF1C2000228821010278
:1034900098210102014B1868704700BF2C0C0022D4
:1034A00010B5044606480BF0CEF93CB1054BD3E805
:1034B000EF1F0139C3E8E21F002AF8D110BD00BF99
:1034C000280C00222C0C00222DE9F041164B054659
:1034D0001B689847154CDFF85880A860444501D315
:1034E000BDE8F08163685B793BB129784B0706D56D
:1034F0002368294620461B6898471034EEE7284683
:103500002E88C1F3C20700F0E9F9C6F3821602461D
:10351000002EEDD00028EBDB01233946204600F0D9
:10352000E5F8B042E9D3E3E7040000228821010274
:1035300098210102044A054B9B1AB1EBD30F34BF0B
:1035400052F8310000207047F82001028821010262
:1035500000200B490B4B30B55B1ADB080A4C0431D9
:103560000133013B00D130BD11F83020256802F055
:10357000070225F007052A4344F8042B0130F0E741
:10358000F82001028821010298030022F8B50646BE
:1035900000240A4F0A4DED1BED08AC4203D14FF059
:1035A000FF342046F8BD57F8340020B13146FDF70E
:1035B000AFFD0028F5D00134EFE700BFF82001028D
:1035C0008821010200282DE9F047884615461F464C
:1035D0001DDA4FF0000A5446DFF8A890254EA6EBFE
:1035E00009063609B24509F1100902D12046BDE8A5
:1035F000F08759F80C0C3B462A4641460079FFF704
:10360000E1FF844238BF04460AF1010AEAE71A4B97
:103610001A4AD21AB5EBD20F29D203EBC5031C7993
:10362000BC4228BF3C4607224FF0090E144EC0B2E0
:1036300000EB400056F82530824023EA020304F0F4
:10364000070282401343032100224EF001E023FAD7
:1036500001F000F00700824238BF024603310FF04C
:103660000BC023F00703134346F82530BEE70024C0
:10367000D9E700BF98210102F82001028821010248
:103680009803002288210102F8B506460F4600245F
:10369000074D084BED1AED08AC4200D3F8BD0021F0
:1036A00022B23B46304601340BF0F2F8A4B2F3E705
:1036B00088210102F820010238B50D4611460A4B57
:1036C0004268C31A1B110446013313714368997190
:1036D000FFF7DAFF012263681D6063685A71BDE875
:1036E00038400BF0CEB800BF8821010210B570B190
:1036F0004168097973B1002A17DBCBB20C4903EB9F
:10370000430351F82200D84000F0070010BD4FF0ED
:10371000FF31EFE70749084C1846641AB2EBD40FA3
:10372000F4D201EBC2010879F0E70420EEE700BF14
:1037300098030022F8200102882101022DE9F04FB0
:1037400087B004AF0446D7E90EA90E4693469846C3
:103750003D6BBAF1000F22D0C7F80490CDF800906D
:103760001021534600207A6BFFF726FAB0F5006F60
:10377000014615D31C490B6813F0060F0BD040F21D
:10378000FF730393194B0222029300231846CDE9DD
:1037900000330BF01CF90C37BD46BDE8F08F5146E5
:1037A00004F007040BF0070BE40044EA8B1444EA2E
:1037B000412444EA055417350D4425F00705ADEBC7
:1037C000050D04ADBAF1000F07D0CDF800905346B7
:1037D0007A6B05F11000FFF7EFF9434622463146B8
:1037E00028460BF085F8D6E7BC030022DD3C010239
:1037F0002DE9F04FC1F34A2691B00D46904607904F
:1038000008930C0D002E5AD000274FF0040B4FF0F8
:103810000A0A0BAB01933A460DAB31464046CDF850
:1038200008B0CDF800A0CDE90D770F97FFF796FB14
:10383000B0F5006FB146034616D325490B6813F067
:10384000060F0ED040F2FF730493D8F80430022222
:103850000393204B3846CDE9017300973B460BF0AC
:10386000B6F811B0BDE8F08FC0F30A0604F11700F6
:10387000184420F00700800809930BF005F866F360
:103880005325044680B1099B00F11001CDE90E37A4
:103890000BABCDE900A30D91404649460E4ACDF849
:1038A00008B00DABFFF75AFB66F353252A462046B6
:1038B000089B079911B0BDE8F04F0BF019B804F15F
:1038C000170020F0070080080AF0DEFF0446EBE74F
:1038D000BC030022153D0102C5E80002436805480B
:1038E000002BA3EB000040F38F0008BF4FF0FF3028
:1038F000704700BF980300220EB403B503AB53F822
:10390000042B01460448019304F0C8FE02B05DF8A0
:1039100004EB03B0704700BFEFE90002CA0605D40C
:103920008B064CBF02490349FFF7E6BF704700BF53
:10393000383F0102543D01022DE9F04F8BB09B4608
:10394000169B9DF854A00693179B04460593189B5D
:103950000D469046199E0493BAF1000F00F09B802B
:1039600006F00103089306F00803079306F480733A
:1039700009930AF08BFF06F002090246074620B1C0
:1039800020468D49FFF7B8FF0746B9F1000F09D06F
:1039900016F0440F32D12A4620468849FFF7ACFF83
:1039A00003461F44089B53B1854B864A53F82A307F
:1039B0002046002B18BF1A468349FFF79DFF099B3D
:1039C000002B48D0079B002B62D14546B8F1000F71
:1039D00005D0424620467D49FFF78EFF0546069BEF
:1039E0003D44002B66D1049B002B6CD1F30700F102
:1039F000DD8031462046FFF791FFD1E0744B186817
:103A000003460028CDD0734B4FF47A791B684FF4EE
:103A10006161B5FBF3F5B5FBF0F300FB135509FB52
:103A200005F5B3FBF1F2B5FBF0FE4FF03C0C01FBEA
:103A3000123100FB1E55B1FBFCF309FB05F5B5FB8C
:103A4000F0F50CFB131120460091CDE901E5624928
:103A5000FFF752FFA4E7079D3DB1604B204653F8A6
:103A60002A205F49FFF748FF0546B8F1000F05D04F
:103A7000424620465549FFF73FFF0544BBF1000F82
:103A8000ADD05A4620465749FFF736FF0544A6E712
:103A90004FF0000BE1E7BBF1010F069B06D1002BB5
:103AA00064D1049B002B7BD000250CE0002BF8D0C8
:103AB0004D485CE04D48069B22464D490AF001FD09
:103AC000049B002B68D0DFF83881DFF83891049F21
:103AD0003146102F204628BF10274FF0000BFFF76C
:103AE0001DFF5D4545DC059B494620461A78FFF7DA
:103AF00003FF4FF0010B1BF0070F03D14146204697
:103B0000FFF7FAFE5F453BD9059B4946204613F86F
:103B10000B20FFF7F1FE0BF1010BBBF1100FEAD107
:103B20004FF0000B20463349FFF7E6FE5A46059B4F
:103B300020469A5CA2F120015F2928BF2E222E493F
:103B4000FFF7DAFE0BF1010BBBF1100F1DD01BF0DC
:103B5000070F03D141462046FFF7CEFE5F455A4688
:103B6000E5D841462046FFF7C7FEEBE71F4855461C
:103B7000A1E741462046FFF7BFFE0BF1010BB0E77E
:103B800020461E49FFF7B8FEC5E7059B3B44059359
:103B9000049BDB1B04939AD1BAF1000F7FF426AF8C
:103BA00020460BB0BDE8F04F0AF04BBF2046054A57
:103BB0000549FFF7A1FE1CE75C3D0102603D0102E3
:103BC000EC2D0102573D01026C410102853D0102CD
:103BD000380C0022340C0022693D0102002E010243
:103BE000893D01028F3D01020BEA0002EFE900026C
:103BF0009D8600029E3D0102764701029A3D010228
:103C00009C3D0102943D01020022012307498842A4
:103C100007D8002A08BF0123054A1360054B186026
:103C20007047012240085B00F1E700BF40420F00EF
:103C3000340C0022380C002238B5134B0D461C689A
:103C4000F4B1124B1A68002A02F10103B8BF012334
:103C5000013B02D16FF0010038BD224612F8101B63
:103C6000814201D01446F3E7E06810B96FF012000A
:103C7000F2E70CF015FE0028F8D000202C60EBE7EE
:103C80006FF00C00E8E700BF08000022142E0102CC
:103C900008B50821024B034A0BF07CF8002008BD50
:103CA000C03D0102C63D010210B5044606F080FF8A
:103CB00008210346074A20460BF06CF82046064AC6
:103CC00008210BF067F82146044808F0D7FA0020D5
:103CD00010BD00BF5B3E01027A3E0102E13C0002E2
:103CE00070B58EB004460D46D0F89C600DF09AF881
:103CF00002460DF03BFF254B25491B589C42254BA6
:103D000018BF0B46101E244A4FF0080108BF10468A
:103D1000224ACDE9004028460BF03CF8D4E90A23BA
:103D2000CDE9022394F90E3028460093237B082125
:103D30001B4A0BF02FF806A92022204607F0B0FD01
:103D4000626E0346009208212846164A0BF022F8BC
:103D5000204605A90DF08AF8034630B1082128460F
:103D6000114A0BF017F80EB070BD6423059A28466F
:103D7000B11A4B43B3FBF6F3CDE90021CDE9026361
:103D800008213346094A0BF005F8ECE71000000063
:103D90009C3D010295520102843E0102873E0102D0
:103DA000933E0102BF3E0102D63E0102033F0102E3
:103DB000F0B50025044693B029460AAF1C220BA893
:103DC0000DF0EEFD134E1A22202138460DF0E8FDCD
:103DD0002146114808F052FA09AA4FF40061304612
:103DE0000DF037F864224FF400630999CDE90057CC
:103DF000C1F500604243D20ACDE90403CDE90231A6
:103E00002046069233460821044A0AF0C3FF28469A
:103E100013B0F0BD78C80022FD3E00023A3F010217
:103E200010B5044606F0E2FE08210346024A204689
:103E30000AF0B0FF002010BD833F01022DE9F341DD
:103E40001746002304460A21B86801AA019301F02D
:103E5000B1FB019DC6B255B12B4601212046144A43
:103E60000AF098FF019D284602B0BDE8F081042EBB
